:1000000003C003C003C003C003C003C003C003C0D8
:1000800016C438C437C436C435C434C433C432C4C7
:1000900031C430C42FC42EC42DC42CC42BC422C0E0
:1000A00040C06CC03EC03DC03CC03BC03AC039C03F
:1000B00038C037C036C035C034C033C0040309046B
:1000C00012011001FF000008D016530703010000C1
:1000D0000001090212000101008032090400000041
:1000E0000000000011241FBECFE5D2E0DEBFCDBF6F
:1000F00000EB0F9307E00F9310E0A0E6B0E0EAEC0E
:10010000FFE102C005900D92A636B107D9F710E0C5
:10011000A6E6B0E001C01D92AA39B107E1F7DFD130
:10012000C1C3BDCFA82FB92F80E090E041E050EAD5
:10013000609530E009C02D9182279795879510F042
:1001400084279527305EC8F36F5FA8F30895EADF30
:100150008D939D930895A6E088279927AA9569F025
:100160000197E1F3B399FCCFB39BFECF81E09927D0
:10017000A6B3019611F0A871D9F70895CF93CFB720
:10018000CF93C0915F02C03B21F4C0915E02C730A3
:1001900021F0CF91CFBFCF9181CFCC27C395B39B17
:1001A000E9F7B39B0BC0B39B09C0B39B07C0B39BDC
:1001B00005C0B39B03C0B39B01C0D3C00F92DF93B4
:1001C000C0917D00DD27CC57DF4F012EB39B03C0CC
:1001D000DF910F90E6CF2F930F931F934F932FEF45
:1001E0004F6F06B303FB20F95F933F9350E03BE072
:1001F00065C016B30126502953FDC89556B3012793
:1002000003FB25F92F7306B3B1F05027102713FB1A
:1002100026F906B22230F0F000C016B3012703FB26
:1002200027F90126502906B22430E8F54F772068D7
:1002300016B30000F6CF50274F7D206206B2102F74
:10024000000000C006B300265029102713FB26F932
:1002500006B2E2CF4F7B06B3206400C0DACF01269E
:100260005029187106B269F14E7F2160012F16B333
:1002700028C0002650294D7F06B22260102F29C0C9
:10028000012650294B7F06B22460012F2DC016B3E2
:1002900001265029477F2860000006B22EC04F7EFD
:1002A00006B3206130C0422706B349930026502987
:1002B000102706B24FEF13FB20F9297F16B379F20E
:1002C000187159F10126502906B2012703FB21F9C3
:1002D000237F06B371F2002650293150D0F006B2C8
:1002E000102713FB22F9277E16B351F2012650295D
:1002F000012703FB06B223F92F7C49F2000006B365
:10030000102713FB24F90026502906B22F7939F261
:1003100070CF10E21ABF002717C03B503195C31BA6
:10032000D04010E21ABF0881033CF9F00B34E9F029
:1003300020917B001981110F1213EDCF093651F175
:100340000D3211F0013E39F7009382003F915F9129
:100350004F911F910F912F91DF910F90CAB7C5FD5B
:100360001DCFCF91CFBFCF9118952091820022232E
:1003700069F310918000112321F5343022F130937C
:10038000800020937C0010917D003BE0311B309376
:100390007D0019C00091800001309CF40AE5309185
:1003A000600034FD11C000936000C0E7D0E010C0D1
:1003B000052710E000C021C0052710E0C89508BB44
:1003C00014C03AE501C032ED032EC0E0D0E032E0C7
:1003D00017B31861C39A08B317BB58E120E84FEF71
:1003E00020FF052708BB279517951C3F28F700001D
:1003F0004552B0F720FF0527279508BB17951C3FEE
:10040000B8F629913A9561F7077E10918100110F96
:1004100008BBC250D04011F010937B0010E21ABF0D
:10042000086017B3177E402F477E54E05A95F1F7C6
:1004300008BB17BB48BB8ACF81E080936700F89464
:10044000E0916E00F0916F00329785E08093570045
:10045000E89507B600FCFDCF789408959C01E091E3
:100460006E00F0916F00309749F1E430F105B1F082
:1004700087E1EC3BF80739F420916A0030916B007A
:100480002E5D3B4F0DC087E1EE3BF80749F420910C
:100490006C0030916D002D5D3B4F02C02FED3BECA9
:1004A000F89481E0090180935700E895112478942D
:1004B0003296F0936F00E0936E00089581E180938F
:1004C0005700E895EBCF8FEF9FEFC8DF80916E006C
:1004D00090916F008F739070892BA9F7ADCF88E151
:1004E0000FB6F89481BD11BC0FBEE0E0F0E085913D
:1004F00094918F5D9B4C39F4E4E0F0E08591949108
:100500008F5D9B4C09F0DFDF10926F0010926E0040
:10051000AC9A8BB780628BBFBB9A88E893E1ECE919
:10052000F1E03197F1F70197D1F7BB987894EE2479
:10053000FF2410918000135017FDD0C080917D00E2
:10054000CCE0D0E0C81BD109CC57DF4F80917C00B4
:100550008D3209F08DC0183009F0BEC083EC809355
:1005600070008AE580936000109269002881822FD4
:1005700080769981882309F1992341F482E690E0FD
:1005800090937F0080937E0024E068C0913051F406
:100590008C819D8190936F0080936E0027FD59C0E0
:1005A0009FEF58C080916600923011F4816001C0C5
:1005B00084608093660020E051C08A8110927900A7
:1005C000992331F410927A0089E790E022E03CC050
:1005D000953019F48093810034C0963011F58B81E9
:1005E000813019F482EE97E104C0823041F484EF47
:1005F00097E190937F0080937E0022E10EC08330CC
:1006000059F48A81882341F48EED97E190937F001D
:1006100080937E0024E001C020E080E480936900A4
:100620001DC0983019F483E890E009C0993019F49E
:100630008093830006C09A3021F489E790E021E09E
:1006400003C089E790E020E090937F0080937E00D4
:1006500005C09E8180E88093690007C08F81882350
:1006600019F49E81921708F0922F9093610034C084
:100670008091690087FF30C080916E0090916F007B
:10068000009739F48881998190936B0080936A0078
:100690000DC08430910539F48881998190936D0063
:1006A00080936C0003C0805C974138F48881998105
:1006B000D5DE125011F02296DFCF80916E0090911E
:1006C0006F008F739070892B39F48091660082607F
:1006D000809366001092610010928000809160000B
:1006E00084FF3CC0809161008F3FC1F1182F893099
:1006F00008F018E0811B809361008091700098E8F9
:100700008927809370001123E1F0E0917E00F09141
:100710007F008091690086FF09C0912FA1E7B0E0BA
:1007200084918D9331969150D9F707C0912FA1E70D
:10073000B0E081918D939150E1F7F0937F00E093C9
:100740007E0081E790E0612F02DD612F6C5F6C30ED
:1007500019F08FEF809361006093600094E186B39D
:10076000887131F49150D9F71092810010927B007A
:1007700010E0992309F411E080916800811739F0A5
:10078000112319F4F8944FD07894109368008CE9F1
:1007900091E00197F1F780916600882319F0EE242B
:1007A000FF2403C00894E11CF11C182F80FF14C023
:1007B000F894E0ECF7E1E054F04083E080935700D8
:1007C000E89507B600FCFDCF3097A9F710926F00AF
:1007D00010926E0078DE789411FF0FC08AE390E2E9
:1007E0000197F1F780916E0090916F008F73907078
:1007F000892B11F068DE01C01FDE12FD08C01092C7
:10080000660080E5E81683ECF80608F492CE82E2F2
:1008100091EA0197F1F7F8941BBE15BA10925F02A6
:1008200010925E023ACCFF920F931F93CF93DF9307
:1008300080E8F82E00E0C0E0D0E0102F1F0D11BFBF
:100840008ADC29E0843392070CF0102FF69421966D
:10085000C830D10511F0012FF0CF115011BF1F5F2B
:10086000012FEC0110C077DC8453994097FF03C03F
:10087000909581959F4F8C179D0714F401B7EC015B
:1008800081B78F5F81BF21B730E0812F90E0019663
:100890008217930744F701BFDF91CF911F910F910A
:1008A000FF900895F894FFCF5AFF17BC400800004E
:1008B0000000000000000000000000000000000038
:1008C00000000000000000000000000000001124F3
:1008D0001FBECFE5D2E0DEBFCDBF10E0A0E6B0E0A6
:1008E000ECE6FBE002C005900D92A236B107D9F705
:1008F0001CD13AC1C5CB05C0EDE1F0E13197F1F76C
:1009000001970097C9F70895AC01407C20E030E0E2
:10091000F901E40FF51F85919491F901EE7FE60F3F
:10092000F71F918380832E5F3F4F2034310581F77D
:100930000895FC01E07C83E080935700E89507B6BA
:1009400000FCFDCF0895CF93DF93EC01A0E0B0E071
:10095000AD014C0F5D1FFB01EA0FFB1F80819181F0
:1009600021E0FA010C0120935700E895112412961A
:10097000A034B10569F785E0FE0180935700E89542
:1009800007B600FCFDCFDF91CF910895DF93CF93A1
:10099000CDB7DEB7C054D0400FB6F894DEBF0FBE5F
:1009A000CDBF209160003091610036952795215090
:1009B0003044FE01319621933193CE018F5B9F4FDE
:1009C000E817F907C1F780E090E0B3DF80E090E03E
:1009D000BE016F5F7F4FB7DFC05CDF4F0FB6F8948B
:1009E000DEBF0FBECDBFCF91DF910895EF92FF9292
:1009F0000F931F93DF93CF93CDB7DEB7C054D04092
:100A00000FB6F894DEBF0FBECDBF00E010E035C0DA
:100A10009B01359527957E010894E11CF11C88E027
:100A2000AE3AB80738F0220F331FE20EF31E8FEFF5
:100A30009FEF07C0FD0185919491220F331FE20EB5
:100A4000F31EF701918380836E5F7F4F12966034AF
:100A50007105F1F68091600090916100800F911F07
:100A600068DF8091600090916100800F911FBE014E
:100A70006F5F7F4F68DF005C1F4FF8E000341F0797
:100A800031F0D801A256BF4F60E070E0C1CFC05C2A
:100A9000DF4F0FB6F894DEBF0FBECDBFCF91DF9111
:100AA0001F910F91FF90EF900895DF93CF93CDB7F3
:100AB000DEB7C054D0400FB6F894DEBF0FBECDBF36
:100AC00080E090E0BE016F5F7F4F1EDF80E090E02E
:100AD000019680329105E1F78FEF9FEF9A8389832A
:100AE00080E090E026DF80E090E0BE016F5F7F4F06
:100AF0002ADFC05CDF4F0FB6F894DEBF0FBECDBF5C
:100B0000CF91DF91089587B3836087BBC19820E0C0
:100B10008DE190E1FC013197F1F7C19A0197F1F76E
:100B2000C1982F5F2A3FA1F7089588B318BA87B3F9
:100B30008FEF87BB8AEF90E0EDE1F0E13197F1F7BD
:100B40000197D1F787B317BA8AEF90E0EDE1F0E1B2
:100B50003197F1F70197D1F7F894A7DF47DF16DF58
:0C0B6000D2DF80E090E00895F894FFCF11
:020B6C00C017B0
:040000030000008079
:00000001FF
